:1000000009C021C020C08EC01EC01DC01CC01BC0A6
:100010001AC019C011241FBECFE9CDBF10E0A4E65D
:10002000B0E001C01D92A237B107E1F710E0A0E6F1
:10003000B0E0EAEFF3E002C005900D92A436B107FC
:10004000D9F7DDD0D8C1DCCFCF92DF92EF92FF920B
:100050000F931F93C82ED62E9A014FEF50E0DED09B
:1000600020916D0030916E0040E050E002D17901A6
:100070008A012D2D30E0DD242C193D09442737FD60
:100080004095542FC801B701CFD02FEF30E040E0AA
:1000900050E0EFD08C2D820F1F910F91FF90EF90C9
:1000A000DF90CF90089563D12CED30E040E050E038
:1000B00002D1862F825E08958091670080936A0046
:1000C0008091680080936B008091690080936C0040
:1000D000EADF80936700E7DF80936800E4DF8093C6
:1000E000690045D1262F862F63E0B7D0E92FF0E0D5
:1000F000E959FF4F1082822F68E7AFD0925E692FD7
:1001000070E080E090E023E930E040E050E08CD007
:100110002AE030E040E050E0CED030936E002093F3
:100120006D0008951F920F920FB60F9211242F9316
:100130003F934F935F936F937F938F939F93AF936F
:10014000BF93CF93DF93EF93FF9380916600882353
:1001500069F5C0916400D091650080916A0060915A
:100160006700AE0171DF80936F0080916B0060913A
:100170006800AE0169DF8093700080916C0060912F
:100180006900AE0161DF809371002196D093650014
:10019000C093640080916D0090916E00C817D907DC
:1001A00028F0109265001092640086DF809166004E
:1001B00091E020916F00281708F490E020917000E2
:1001C000281708F0926020917100281708F09460B9
:1001D00098BB8F5F80936600FF91EF91DF91CF9185
:1001E000BF91AF919F918F917F916F915F914F914F
:1001F0003F912F910F900FBE0F901F901895109266
:100200006700109268001092690056DF8FEF87BB7D
:1002100081E083BF82E089BF7894FFCFBA0188274D
:1002200099274427552700C0FF27EE27BB27AA2779
:1002300060FF04C0A20FB31FE41FF51F220F331F7E
:10024000441F551F969587957795679589F7009771
:10025000760771F7CF01BD010895991B79E004C0BD
:10026000991F961708F0961B881F7A95C9F78095F5
:100270000895A1E21A2EAA1BBB1BFD010DC0AA1FE7
:10028000BB1FEE1FFF1FA217B307E407F50720F0FF
:10029000A21BB30BE40BF50B661F771F881F991F7A
:1002A0001A9469F760957095809590959B01AC01C3
:1002B000BD01CF01089597FB092E05260ED057FDED
:1002C00004D0D7DF0AD0001C38F450954095309503
:1002D00021953F4F4F4F5F4F0895F6F790958095CA
:1002E000709561957F4F8F4F9F4F0895A0E0B0E0CC
:1002F000EBE7F1E051C0EC01688179818A819B8153
:10030000611571058105910521F464E279ED8BE5B4
:1003100097E02DE133EF41E050E0CDDF79018A0134
:1003200027EA31E440E050E07FDF5B016C01C80167
:10033000B7012CEE34EF4FEF5FEF76DF9B01AC019E
:100340002A0D3B1D4C1D5D1D57FF04C02150304040
:1003500040405048288339834A835B835F77B901E3
:10036000CA01CDB7DEB7EAE033C0C0DF089580E64A
:1003700090E0BCDF0895609360007093610080930B
:1003800062009093630008952F923F924F925F9284
:100390006F927F928F929F92AF92BF92CF92DF9295
:1003A000EF92FF920F931F93CF93DF93CDB7DEB7FA
:1003B000CA1BDB0B0FB6F894DEBF0FBECDBF09948E
:1003C0002A88398848885F846E847D848C849B84E5
:1003D000AA84B984C884DF80EE80FD800C811B81F3
:1003E000AA81B981CE0FD11D0FB6F894DEBF0FBE22
:0A03F000CDBFED010895F894FFCF92
:0403FA0001000000FE
:00000001FF
